 verify

 Timestamp is 9f65ea12 (reproducible build file hash)

 Preferred load address is 10000000

 Start         Length     Name                   Class
 0001:00000000 00005515H .text$mn                CODE
 0002:00000000 00000124H .idata$5                DATA
 0002:00000124 00000008H .00cfg                  DATA
 0002:0000012c 00000004H .CRT$XCA                DATA
 0002:00000130 00000004H .CRT$XCZ                DATA
 0002:00000134 00000004H .CRT$XIA                DATA
 0002:00000138 00000004H .CRT$XIZ                DATA
 0002:0000013c 00000004H .CRT$XPA                DATA
 0002:00000140 00000004H .CRT$XPZ                DATA
 0002:00000144 00000004H .CRT$XTA                DATA
 0002:00000148 00000008H .CRT$XTZ                DATA
 0002:0000014c 00000000H .gfids$y                DATA
 0002:00000150 00001670H .rdata                  DATA
 0002:000017c0 00000000H .rdata$CastGuardVftablesA DATA
 0002:000017c0 00000000H .rdata$CastGuardVftablesC DATA
 0002:000017c0 00000004H .rdata$sxdata           DATA
 0002:000017c4 00000064H .rdata$voltmd           DATA
 0002:00001828 0000029cH .rdata$zzzdbg           DATA
 0002:00001ac4 00000004H .rtc$IAA                DATA
 0002:00001ac8 00000004H .rtc$IZZ                DATA
 0002:00001acc 00000004H .rtc$TAA                DATA
 0002:00001ad0 00000008H .rtc$TZZ                DATA
 0002:00001ad8 00000088H .xdata$x                DATA
 0002:00001b60 00000058H .edata                  DATA
 0002:00001bb8 00000078H .idata$2                DATA
 0002:00001c30 00000014H .idata$3                DATA
 0002:00001c44 00000124H .idata$4                DATA
 0002:00001d68 0000070cH .idata$6                DATA
 0003:00000000 000000e8H .data                   DATA
 0003:000000e8 0000036cH .bss                    DATA
 0004:00000000 00000060H .rsrc$01                DATA
 0004:00000060 00000328H .rsrc$02                DATA

  Address         Publics by Value              Rva+Base       Lib:Object

 0000:00000000       ___AbsoluteZero            00000000     <absolute>
 0000:00000000       ___arm64x_extra_rfe_table  00000000     <absolute>
 0000:00000000       ___arm64x_extra_rfe_table_size 00000000     <absolute>
 0000:00000000       ___arm64x_native_entrypoint 00000000     <absolute>
 0000:00000000       ___arm64x_redirection_metadata 00000000     <absolute>
 0000:00000000       ___arm64x_redirection_metadata_count 00000000     <absolute>
 0000:00000000       ___dynamic_value_reloc_table 00000000     <absolute>
 0000:00000000       ___enclave_config          00000000     <absolute>
 0000:00000000       ___guard_check_icall_a64n_fptr 00000000     <absolute>
 0000:00000000       ___guard_eh_cont_count     00000000     <absolute>
 0000:00000000       ___guard_eh_cont_table     00000000     <absolute>
 0000:00000000       ___guard_fids_count        00000000     <absolute>
 0000:00000000       ___guard_fids_table        00000000     <absolute>
 0000:00000000       ___guard_iat_count         00000000     <absolute>
 0000:00000000       ___guard_iat_table         00000000     <absolute>
 0000:00000000       ___guard_longjmp_count     00000000     <absolute>
 0000:00000000       ___guard_longjmp_table     00000000     <absolute>
 0000:00000000       ___hybrid_auxiliary_delayload_iat 00000000     <absolute>
 0000:00000000       ___hybrid_auxiliary_delayload_iat_copy 00000000     <absolute>
 0000:00000000       ___hybrid_auxiliary_iat    00000000     <absolute>
 0000:00000000       ___hybrid_auxiliary_iat_copy 00000000     <absolute>
 0000:00000000       ___hybrid_code_map         00000000     <absolute>
 0000:00000000       ___hybrid_code_map_count   00000000     <absolute>
 0000:00000000       ___hybrid_image_info_bitfield 00000000     <absolute>
 0000:00000000       ___x64_code_ranges_to_entry_points 00000000     <absolute>
 0000:00000000       ___x64_code_ranges_to_entry_points_count 00000000     <absolute>
 0000:00000001       ___safe_se_handler_count   00000001     <absolute>
 0000:00000100       ___guard_flags             00000100     <absolute>
 0000:00000000       ___ImageBase               10000000     <linker-defined>
 0001:0000019e       _VerifyClassForMajorVersion 1000119e f   check_code.obj
 0001:00000cd2       _initialize_class_hash     10001cd2 f   check_code.obj
 0001:00004640       _jio_vsnprintf             10005640 f   jvm:jvm.dll
 0001:00004646       _jio_snprintf              10005646 f   jvm:jvm.dll
 0001:0000464c       _JVM_FindClassFromClass@16 1000564c f   jvm:jvm.dll
 0001:00004652       _JVM_IsInterface@8         10005652 f   jvm:jvm.dll
 0001:00004658       _JVM_GetClassNameUTF@8     10005658 f   jvm:jvm.dll
 0001:0000465e       _JVM_GetClassCPTypes@12    1000565e f   jvm:jvm.dll
 0001:00004664       _JVM_GetClassCPEntriesCount@8 10005664 f   jvm:jvm.dll
 0001:0000466a       _JVM_GetClassFieldsCount@8 1000566a f   jvm:jvm.dll
 0001:00004670       _JVM_GetClassMethodsCount@8 10005670 f   jvm:jvm.dll
 0001:00004676       _JVM_GetMethodIxExceptionIndexes@16 10005676 f   jvm:jvm.dll
 0001:0000467c       _JVM_GetMethodIxExceptionsCount@12 1000567c f   jvm:jvm.dll
 0001:00004682       _JVM_GetMethodIxByteCode@16 10005682 f   jvm:jvm.dll
 0001:00004688       _JVM_GetMethodIxByteCodeLength@12 10005688 f   jvm:jvm.dll
 0001:0000468e       _JVM_GetMethodIxExceptionTableEntry@20 1000568e f   jvm:jvm.dll
 0001:00004694       _JVM_GetMethodIxExceptionTableLength@12 10005694 f   jvm:jvm.dll
 0001:0000469a       _JVM_GetFieldIxModifiers@12 1000569a f   jvm:jvm.dll
 0001:000046a0       _JVM_GetMethodIxModifiers@12 100056a0 f   jvm:jvm.dll
 0001:000046a6       _JVM_GetMethodIxLocalsCount@12 100056a6 f   jvm:jvm.dll
 0001:000046ac       _JVM_GetMethodIxArgsSize@12 100056ac f   jvm:jvm.dll
 0001:000046b2       _JVM_GetMethodIxMaxStack@12 100056b2 f   jvm:jvm.dll
 0001:000046b8       _JVM_IsConstructorIx@12    100056b8 f   jvm:jvm.dll
 0001:000046be       _JVM_IsVMGeneratedMethodIx@12 100056be f   jvm:jvm.dll
 0001:000046c4       _JVM_GetMethodIxNameUTF@12 100056c4 f   jvm:jvm.dll
 0001:000046ca       _JVM_GetMethodIxSignatureUTF@12 100056ca f   jvm:jvm.dll
 0001:000046d0       _JVM_GetCPMethodNameUTF@12 100056d0 f   jvm:jvm.dll
 0001:000046d6       _JVM_GetCPMethodSignatureUTF@12 100056d6 f   jvm:jvm.dll
 0001:000046dc       _JVM_GetCPFieldSignatureUTF@12 100056dc f   jvm:jvm.dll
 0001:000046e2       _JVM_GetCPClassNameUTF@12  100056e2 f   jvm:jvm.dll
 0001:000046e8       _JVM_GetCPFieldClassNameUTF@12 100056e8 f   jvm:jvm.dll
 0001:000046ee       _JVM_GetCPMethodClassNameUTF@12 100056ee f   jvm:jvm.dll
 0001:000046f4       _JVM_GetCPFieldModifiers@16 100056f4 f   jvm:jvm.dll
 0001:000046fa       _JVM_GetCPMethodModifiers@16 100056fa f   jvm:jvm.dll
 0001:00004700       _JVM_ReleaseUTF@4          10005700 f   jvm:jvm.dll
 0001:00004706       _JVM_IsSameClassPackage@12 10005706 f   jvm:jvm.dll
 0001:0000470c       ___raise_securityfailure   1000570c f   MSVCRT:gs_report.obj
 0001:00004734       ___report_gsfailure        10005734 f   MSVCRT:gs_report.obj
 0001:0000482e       ___report_rangecheckfailure 1000582e f   MSVCRT:gs_report.obj
 0001:0000483a       ___report_securityfailure  1000583a f   MSVCRT:gs_report.obj
 0001:00004909       @__security_check_cookie@4 10005909 f   MSVCRT:secchk.obj
 0001:00004c57       __DllMainCRTStartup@12     10005c57 f   MSVCRT:dll_dllmain.obj
 0001:00004cc7       ___security_init_cookie    10005cc7 f   MSVCRT:gs_support.obj
 0001:00004d12       _DllMain@12                10005d12 f   MSVCRT:dll_dllmain_stub.obj
 0001:00004d34       ?__scrt_initialize_type_info@@YAXXZ 10005d34 f   MSVCRT:tncleanup.obj
 0001:00004d40       ?__scrt_uninitialize_type_info@@YAXXZ 10005d40 f   MSVCRT:tncleanup.obj
 0001:00004d4c       ___local_stdio_printf_options 10005d4c f i MSVCRT:default_local_stdio_options.obj
 0001:00004d52       ___local_stdio_scanf_options 10005d52 f i MSVCRT:default_local_stdio_options.obj
 0001:00004d58       ___scrt_initialize_default_local_stdio_options 10005d58 f   MSVCRT:default_local_stdio_options.obj
 0001:00004db9       ___scrt_acquire_startup_lock 10005db9 f   MSVCRT:utility.obj
 0001:00004deb       ___scrt_dllmain_after_initialize_c 10005deb f   MSVCRT:utility.obj
 0001:00004e16       ___scrt_dllmain_before_initialize_c 10005e16 f   MSVCRT:utility.obj
 0001:00004e24       ___scrt_dllmain_crt_thread_attach 10005e24 f   MSVCRT:utility.obj
 0001:00004e43       ___scrt_dllmain_crt_thread_detach 10005e43 f   MSVCRT:utility.obj
 0001:00004e50       ___scrt_dllmain_exception_filter 10005e50 f   MSVCRT:utility.obj
 0001:00004e84       ___scrt_dllmain_uninitialize_c 10005e84 f   MSVCRT:utility.obj
 0001:00004ea7       ___scrt_dllmain_uninitialize_critical 10005ea7 f   MSVCRT:utility.obj
 0001:00004eb4       ___scrt_initialize_crt     10005eb4 f   MSVCRT:utility.obj
 0001:00004eed       ___scrt_initialize_onexit_tables 10005eed f   MSVCRT:utility.obj
 0001:00004f74       ___scrt_is_nonwritable_in_current_image 10005f74 f   MSVCRT:utility.obj
 0001:00005008       ___scrt_release_startup_lock 10006008 f   MSVCRT:utility.obj
 0001:00005025       ___scrt_uninitialize_crt   10006025 f   MSVCRT:utility.obj
 0001:0000504d       ___scrt_get_dyn_tls_init_callback 1000604d f   MSVCRT:dyn_tls_init.obj
 0001:00005053       ___scrt_fastfail           10006053 f   MSVCRT:utility_desktop.obj
 0001:0000516e       __crt_debugger_hook        1000616e f   MSVCRT:utility_desktop.obj
 0001:00005176       __RTC_Initialize           10006176 f   MSVCRT:initsect.obj
 0001:000051a2       __RTC_Terminate            100061a2 f   MSVCRT:initsect.obj
 0001:000051d0       __SEH_prolog4              100061d0 f   MSVCRT:sehprolg4.obj
 0001:00005215       __except_handler4          10006215 f   MSVCRT:chandler4gs.obj
 0001:00005244       @_guard_check_icall_nop@4  10006244 f i MSVCRT:guard_support.obj
 0001:00005247       ___isa_available_init      10006247 f   MSVCRT:cpu_disp.obj
 0001:0000541b       __get_startup_argv_mode    1000641b f   MSVCRT:argv_mode.obj
 0001:0000541f       ___scrt_is_ucrt_dll_in_use 1000641f f   MSVCRT:ucrt_detection.obj
 0001:0000542b       _memcpy                    1000642b f   vcruntime:VCRUNTIME140.dll
 0001:00005431       _memset                    10006431 f   vcruntime:VCRUNTIME140.dll
 0001:00005437       _strchr                    10006437 f   vcruntime:VCRUNTIME140.dll
 0001:0000543d       _longjmp                   1000643d f   vcruntime:VCRUNTIME140.dll
 0001:00005443       __setjmp3                  10006443 f   vcruntime:VCRUNTIME140.dll
 0001:00005449       ___std_type_info_destroy_list 10006449 f   vcruntime:VCRUNTIME140.dll
 0001:0000544f       __except_handler4_common   1000644f f   vcruntime:VCRUNTIME140.dll
 0001:00005455       _strcmp                    10006455 f   ucrt:api-ms-win-crt-string-l1-1-0.dll
 0001:0000545b       _strcpy                    1000645b f   ucrt:api-ms-win-crt-string-l1-1-0.dll
 0001:00005461       _strlen                    10006461 f   ucrt:api-ms-win-crt-string-l1-1-0.dll
 0001:00005467       __initterm                 10006467 f   ucrt:api-ms-win-crt-runtime-l1-1-0.dll
 0001:0000546d       __initterm_e               1000646d f   ucrt:api-ms-win-crt-runtime-l1-1-0.dll
 0001:00005473       __seh_filter_dll           10006473 f   ucrt:api-ms-win-crt-runtime-l1-1-0.dll
 0001:00005479       __configure_narrow_argv    10006479 f   ucrt:api-ms-win-crt-runtime-l1-1-0.dll
 0001:0000547f       __initialize_narrow_environment 1000647f f   ucrt:api-ms-win-crt-runtime-l1-1-0.dll
 0001:00005485       __initialize_onexit_table  10006485 f   ucrt:api-ms-win-crt-runtime-l1-1-0.dll
 0001:0000548b       __execute_onexit_table     1000648b f   ucrt:api-ms-win-crt-runtime-l1-1-0.dll
 0001:00005491       __cexit                    10006491 f   ucrt:api-ms-win-crt-runtime-l1-1-0.dll
 0001:00005497       ___acrt_initialize         10006497 f   MSVCRT:ucrt_stubs.obj
 0001:00005497       ___acrt_thread_attach      10006497 f   MSVCRT:ucrt_stubs.obj
 0001:00005497       ___acrt_thread_detach      10006497 f   MSVCRT:ucrt_stubs.obj
 0001:00005497       ___acrt_uninitialize       10006497 f   MSVCRT:ucrt_stubs.obj
 0001:00005497       ___acrt_uninitialize_critical 10006497 f   MSVCRT:ucrt_stubs.obj
 0001:00005497       ___scrt_stub_for_acrt_initialize 10006497 f   MSVCRT:ucrt_stubs.obj
 0001:00005497       ___scrt_stub_for_acrt_thread_attach 10006497 f   MSVCRT:ucrt_stubs.obj
 0001:00005497       ___scrt_stub_for_acrt_thread_detach 10006497 f   MSVCRT:ucrt_stubs.obj
 0001:00005497       ___scrt_stub_for_acrt_uninitialize 10006497 f   MSVCRT:ucrt_stubs.obj
 0001:00005497       ___scrt_stub_for_acrt_uninitialize_critical 10006497 f   MSVCRT:ucrt_stubs.obj
 0001:00005497       ___vcrt_initialize         10006497 f   MSVCRT:ucrt_stubs.obj
 0001:00005497       ___vcrt_thread_attach      10006497 f   MSVCRT:ucrt_stubs.obj
 0001:00005497       ___vcrt_thread_detach      10006497 f   MSVCRT:ucrt_stubs.obj
 0001:00005497       ___vcrt_uninitialize       10006497 f   MSVCRT:ucrt_stubs.obj
 0001:00005497       ___vcrt_uninitialize_critical 10006497 f   MSVCRT:ucrt_stubs.obj
 0001:0000549a       ___scrt_stub_for_is_c_termination_complete 1000649a f   MSVCRT:ucrt_stubs.obj
 0001:0000549a       __is_c_termination_complete 1000649a f   MSVCRT:ucrt_stubs.obj
 0001:0000549d       __filter_x86_sse2_floating_point_exception 1000649d f   MSVCRT:x86_exception_filter.obj
 0001:0000549d       __filter_x86_sse2_floating_point_exception_default 1000649d f   MSVCRT:x86_exception_filter.obj
 0002:00000000       __imp__QueryPerformanceCounter@4 10007000     kernel32:KERNEL32.dll
 0002:00000004       __imp__IsProcessorFeaturePresent@4 10007004     kernel32:KERNEL32.dll
 0002:00000008       __imp__TerminateProcess@8  10007008     kernel32:KERNEL32.dll
 0002:0000000c       __imp__GetCurrentProcess@0 1000700c     kernel32:KERNEL32.dll
 0002:00000010       __imp__SetUnhandledExceptionFilter@4 10007010     kernel32:KERNEL32.dll
 0002:00000014       __imp__UnhandledExceptionFilter@4 10007014     kernel32:KERNEL32.dll
 0002:00000018       __imp__GetCurrentThreadId@0 10007018     kernel32:KERNEL32.dll
 0002:0000001c       __imp__GetSystemTimeAsFileTime@4 1000701c     kernel32:KERNEL32.dll
 0002:00000020       __imp__DisableThreadLibraryCalls@4 10007020     kernel32:KERNEL32.dll
 0002:00000024       __imp__InitializeSListHead@4 10007024     kernel32:KERNEL32.dll
 0002:00000028       __imp__IsDebuggerPresent@0 10007028     kernel32:KERNEL32.dll
 0002:0000002c       __imp__GetCurrentProcessId@0 1000702c     kernel32:KERNEL32.dll
 0002:00000030       \177KERNEL32_NULL_THUNK_DATA 10007030     kernel32:KERNEL32.dll
 0002:00000034       __imp__memcpy              10007034     vcruntime:VCRUNTIME140.dll
 0002:00000038       __imp__memset              10007038     vcruntime:VCRUNTIME140.dll
 0002:0000003c       __imp__strchr              1000703c     vcruntime:VCRUNTIME140.dll
 0002:00000040       __imp___except_handler4_common 10007040     vcruntime:VCRUNTIME140.dll
 0002:00000044       __imp____std_type_info_destroy_list 10007044     vcruntime:VCRUNTIME140.dll
 0002:00000048       __imp___setjmp3            10007048     vcruntime:VCRUNTIME140.dll
 0002:0000004c       __imp__longjmp             1000704c     vcruntime:VCRUNTIME140.dll
 0002:00000050       \177VCRUNTIME140_NULL_THUNK_DATA 10007050     vcruntime:VCRUNTIME140.dll
 0002:00000054       __imp__free                10007054     ucrt:api-ms-win-crt-heap-l1-1-0.dll
 0002:00000058       __imp__malloc              10007058     ucrt:api-ms-win-crt-heap-l1-1-0.dll
 0002:0000005c       __imp__calloc              1000705c     ucrt:api-ms-win-crt-heap-l1-1-0.dll
 0002:00000060       \177api-ms-win-crt-heap-l1-1-0_NULL_THUNK_DATA 10007060     ucrt:api-ms-win-crt-heap-l1-1-0.dll
 0002:00000064       __imp___seh_filter_dll     10007064     ucrt:api-ms-win-crt-runtime-l1-1-0.dll
 0002:00000068       __imp___configure_narrow_argv 10007068     ucrt:api-ms-win-crt-runtime-l1-1-0.dll
 0002:0000006c       __imp___initialize_narrow_environment 1000706c     ucrt:api-ms-win-crt-runtime-l1-1-0.dll
 0002:00000070       __imp___initialize_onexit_table 10007070     ucrt:api-ms-win-crt-runtime-l1-1-0.dll
 0002:00000074       __imp___execute_onexit_table 10007074     ucrt:api-ms-win-crt-runtime-l1-1-0.dll
 0002:00000078       __imp___cexit              10007078     ucrt:api-ms-win-crt-runtime-l1-1-0.dll
 0002:0000007c       __imp___initterm           1000707c     ucrt:api-ms-win-crt-runtime-l1-1-0.dll
 0002:00000080       __imp___initterm_e         10007080     ucrt:api-ms-win-crt-runtime-l1-1-0.dll
 0002:00000084       \177api-ms-win-crt-runtime-l1-1-0_NULL_THUNK_DATA 10007084     ucrt:api-ms-win-crt-runtime-l1-1-0.dll
 0002:00000088       __imp__strcpy              10007088     ucrt:api-ms-win-crt-string-l1-1-0.dll
 0002:0000008c       __imp__strlen              1000708c     ucrt:api-ms-win-crt-string-l1-1-0.dll
 0002:00000090       __imp__strcmp              10007090     ucrt:api-ms-win-crt-string-l1-1-0.dll
 0002:00000094       \177api-ms-win-crt-string-l1-1-0_NULL_THUNK_DATA 10007094     ucrt:api-ms-win-crt-string-l1-1-0.dll
 0002:00000098       __imp__JVM_GetCPFieldModifiers@16 10007098     jvm:jvm.dll
 0002:0000009c       __imp__JVM_GetCPMethodClassNameUTF@12 1000709c     jvm:jvm.dll
 0002:000000a0       __imp__JVM_GetCPFieldClassNameUTF@12 100070a0     jvm:jvm.dll
 0002:000000a4       __imp__JVM_GetCPClassNameUTF@12 100070a4     jvm:jvm.dll
 0002:000000a8       __imp__JVM_GetCPFieldSignatureUTF@12 100070a8     jvm:jvm.dll
 0002:000000ac       __imp__JVM_GetCPMethodSignatureUTF@12 100070ac     jvm:jvm.dll
 0002:000000b0       __imp__JVM_GetCPMethodNameUTF@12 100070b0     jvm:jvm.dll
 0002:000000b4       __imp__JVM_GetMethodIxSignatureUTF@12 100070b4     jvm:jvm.dll
 0002:000000b8       __imp__JVM_GetMethodIxNameUTF@12 100070b8     jvm:jvm.dll
 0002:000000bc       __imp__JVM_IsVMGeneratedMethodIx@12 100070bc     jvm:jvm.dll
 0002:000000c0       __imp__JVM_IsConstructorIx@12 100070c0     jvm:jvm.dll
 0002:000000c4       __imp__JVM_GetMethodIxMaxStack@12 100070c4     jvm:jvm.dll
 0002:000000c8       __imp__JVM_GetMethodIxArgsSize@12 100070c8     jvm:jvm.dll
 0002:000000cc       __imp__JVM_GetMethodIxLocalsCount@12 100070cc     jvm:jvm.dll
 0002:000000d0       __imp__JVM_ReleaseUTF@4    100070d0     jvm:jvm.dll
 0002:000000d4       __imp__jio_vsnprintf       100070d4     jvm:jvm.dll
 0002:000000d8       __imp__JVM_IsSameClassPackage@12 100070d8     jvm:jvm.dll
 0002:000000dc       __imp__JVM_GetMethodIxModifiers@12 100070dc     jvm:jvm.dll
 0002:000000e0       __imp__JVM_GetFieldIxModifiers@12 100070e0     jvm:jvm.dll
 0002:000000e4       __imp__JVM_GetMethodIxExceptionTableLength@12 100070e4     jvm:jvm.dll
 0002:000000e8       __imp__JVM_GetMethodIxExceptionTableEntry@20 100070e8     jvm:jvm.dll
 0002:000000ec       __imp__JVM_GetMethodIxByteCodeLength@12 100070ec     jvm:jvm.dll
 0002:000000f0       __imp__JVM_GetMethodIxByteCode@16 100070f0     jvm:jvm.dll
 0002:000000f4       __imp__JVM_GetMethodIxExceptionsCount@12 100070f4     jvm:jvm.dll
 0002:000000f8       __imp__JVM_GetMethodIxExceptionIndexes@16 100070f8     jvm:jvm.dll
 0002:000000fc       __imp__JVM_GetClassMethodsCount@8 100070fc     jvm:jvm.dll
 0002:00000100       __imp__JVM_GetClassFieldsCount@8 10007100     jvm:jvm.dll
 0002:00000104       __imp__JVM_GetClassCPEntriesCount@8 10007104     jvm:jvm.dll
 0002:00000108       __imp__JVM_GetClassCPTypes@12 10007108     jvm:jvm.dll
 0002:0000010c       __imp__JVM_GetClassNameUTF@8 1000710c     jvm:jvm.dll
 0002:00000110       __imp__JVM_IsInterface@8   10007110     jvm:jvm.dll
 0002:00000114       __imp__JVM_FindClassFromClass@16 10007114     jvm:jvm.dll
 0002:00000118       __imp__JVM_GetCPMethodModifiers@16 10007118     jvm:jvm.dll
 0002:0000011c       __imp__jio_snprintf        1000711c     jvm:jvm.dll
 0002:00000120       \177jvm_NULL_THUNK_DATA    10007120     jvm:jvm.dll
 0002:00000124       ___guard_check_icall_fptr  10007124     MSVCRT:guard_support.obj
 0002:00000128       ___castguard_check_failure_os_handled_fptr 10007128     MSVCRT:guard_support.obj
 0002:0000012c       ___xc_a                    1000712c     MSVCRT:initializers.obj
 0002:00000130       ___xc_z                    10007130     MSVCRT:initializers.obj
 0002:00000134       ___xi_a                    10007134     MSVCRT:initializers.obj
 0002:00000138       ___xi_z                    10007138     MSVCRT:initializers.obj
 0002:0000013c       ___xp_a                    1000713c     MSVCRT:initializers.obj
 0002:00000140       ___xp_z                    10007140     MSVCRT:initializers.obj
 0002:00000144       ___xt_a                    10007144     MSVCRT:initializers.obj
 0002:00000148       ___xt_z                    10007148     MSVCRT:initializers.obj
 0002:00000150       _opcode_in_out             10007150     check_code.obj
 0002:00000880       ??_C@_00CNPNBAHC@@         10007880     check_code.obj
 0002:00000884       ??_C@_01FHEEJDEE@A@        10007884     check_code.obj
 0002:00000888       ??_C@_01JPJNBJEM@I@        10007888     check_code.obj
 0002:0000088c       ??_C@_01OCOKONAJ@L@        1000788c     check_code.obj
 0002:00000890       ??_C@_01BIAFAFID@F@        10007890     check_code.obj
 0002:00000894       ??_C@_01CKDDGHAB@D@        10007894     check_code.obj
 0002:00000898       ??_C@_01OGPIMHDM@?$DP@     10007898     check_code.obj
 0002:0000089c       ??_C@_04NFNNKICA@?$FLI?$FNI@ 1000789c     check_code.obj
 0002:000008a4       ??_C@_04OCADFIBC@?$FLL?$FNI@ 100078a4     check_code.obj
 0002:000008ac       ??_C@_04INLOLIHG@?$FLF?$FNI@ 100078ac     check_code.obj
 0002:000008b4       ??_C@_04CHLHHAPN@?$FLD?$FNI@ 100078b4     check_code.obj
 0002:000008bc       ??_C@_04BAGJIAMP@?$FLA?$FNI@ 100078bc     check_code.obj
 0002:000008c4       ??_C@_04CNMCPCB@?$FLB?$FNI@ 100078c4     check_code.obj
 0002:000008cc       ??_C@_04LKGAEIEE@?$FLC?$FNI@ 100078cc     check_code.obj
 0002:000008d4       ??_C@_04OKHJBPNL@?$FLS?$FNI@ 100078d4     check_code.obj
 0002:000008dc       ??_C@_05BKAAAJCM@?$FLI?$FNII@ 100078dc     check_code.obj
 0002:000008e4       ??_C@_05KPJHHCBJ@?$FLL?$FNIL@ 100078e4     check_code.obj
 0002:000008ec       ??_C@_05BPMIICDC@?$FLF?$FNIF@ 100078ec     check_code.obj
 0002:000008f4       ??_C@_05FHDOLDNA@?$FLD?$FNID@ 100078f4     check_code.obj
 0002:000008fc       ??_C@_05OCKJMIOF@?$FLA?$FNIA@ 100078fc     check_code.obj
 0002:00000904       ??_C@_05GNNADIDN@?$FLB?$FNII@ 10007904     check_code.obj
 0002:0000090c       ??_C@_05FALABBIN@?$FLC?$FNII@ 1000790c     check_code.obj
 0002:00000914       ??_C@_05DAFAIGAP@?$FLS?$FNII@ 10007914     check_code.obj
 0002:0000091c       ??_C@_01HIHLOKLC@1@        1000791c     check_code.obj
 0002:00000920       ??_C@_03HGNMLOHK@2?$CL1@   10007920     check_code.obj
 0002:00000924       ??_C@_02ODEKKOPI@11@       10007924     check_code.obj
 0002:00000928       ??_C@_02OBAMBAKB@21@       10007928     check_code.obj
 0002:0000092c       ??_C@_03HHJOIJGL@121@      1000792c     check_code.obj
 0002:00000930       ??_C@_04EJNNNEMH@3?$CL21@  10007930     check_code.obj
 0002:00000938       ??_C@_04KGLAPINH@1321@     10007938     check_code.obj
 0002:00000940       ??_C@_04ELBJEKIM@2121@     10007940     check_code.obj
 0002:00000948       ??_C@_04HHDLFECN@32?$CL1@  10007948     check_code.obj
 0002:00000950       ??_C@_05JIOCAIMP@21321@    10007950     check_code.obj
 0002:00000958       ??_C@_06BNDCAIPK@4?$CL32?$CL1@ 10007958     check_code.obj
 0002:00000960       ??_C@_06MFMEDPLH@214321@   10007960     check_code.obj
 0002:00000968       ??_C@_02MIGHPNDL@12@       10007968     check_code.obj
 0002:0000096c       ??_C@_02FOEOGEOO@II@       1000796c     check_code.obj
 0002:00000970       ??_C@_02CFPCFCEA@LL@       10007970     check_code.obj
 0002:00000974       ??_C@_02NCIKDPBM@FF@       10007974     check_code.obj
 0002:00000978       ??_C@_02ODDIIJPA@DD@       10007978     check_code.obj
 0002:0000097c       ??_C@_02FIIFKGAF@LI@       1000797c     check_code.obj
 0002:00000980       ??_C@_02JIIELPFO@AA@       10007980     check_code.obj
 0002:00000984       ??_C@_01DGKLNCNG@R@        10007984     check_code.obj
 0002:00000988       ??_C@_03OCJFCJPE@?$FL?$DP?$FN@ 10007988     check_code.obj
 0002:0000098c       ??_C@_01MJMHLOMK@O@        1000798c     check_code.obj
 0002:00000990       ??_C@_01IDAFKMJL@_@        10007990     check_code.obj
 0002:00000994       ??_C@_0BF@LJMGCLHE@Cannot?5find?5class?5?$CFs@ 10007994     check_code.obj
 0002:000009ac       ??_C@_0BB@DDFKOHA@java?1lang?1Object@ 100079ac     check_code.obj
 0002:000009c0       ??_C@_0BB@FLFAIHG@java?1lang?1String@ 100079c0     check_code.obj
 0002:000009d4       ??_C@_0BE@ILKHHCBH@java?1lang?1Throwable@ 100079d4     check_code.obj
 0002:000009e8       ??_C@_0BE@BMOODFFE@java?1lang?1Cloneable@ 100079e8     check_code.obj
 0002:000009fc       ??_C@_0BF@KBKNMCMB@java?1io?1Serializable@ 100079fc     check_code.obj
 0002:00000a14       ??_C@_0BK@GOGHCOEH@Inconsistent?5access?5bits?4@ 10007a14     check_code.obj
 0002:00000a30       ??_C@_0CH@BFIAKBBO@Illegal?5instruction?5found?5at?5of@ 10007a30     check_code.obj
 0002:00000a58       ??_C@_0DP@NHEDEPNH@Code?5stops?5in?5the?5middle?5of?5ins@ 10007a58     check_code.obj
 0002:00000a98       ??_C@_0L@FLBIKONJ@Empty?5code@ 10007a98     check_code.obj
 0002:00000aa4       ??_C@_0CB@FKJLIIBN@Illegal?5target?5of?5jump?5or?5branc@ 10007aa4     check_code.obj
 0002:00000ac8       ??_C@_0CB@GILFIHLF@Non?5zero?5padding?5bytes?5in?5switc@ 10007ac8     check_code.obj
 0002:00000aec       ??_C@_0BH@FEOHEHFA@Unsorted?5lookup?5switch@ 10007aec     check_code.obj
 0002:00000b04       ??_C@_0CB@BKGPDLNL@Illegal?5default?5target?5in?5switc@ 10007b04     check_code.obj
 0002:00000b28       ??_C@_0BO@OAIMDCHG@Illegal?5branch?5in?5tableswitch@ 10007b28     check_code.obj
 0002:00000b48       ??_C@_06FALKBLGB@?$DMinit?$DO@ 10007b48     check_code.obj
 0002:00000b50       ??_C@_0CL@PDOJFDFJ@Must?5call?5initializers?5using?5in@ 10007b50     check_code.obj
 0002:00000b7c       ??_C@_0CA@IPAEHINF@Illegal?5call?5to?5internal?5method@ 10007b7c     check_code.obj
 0002:00000b9c       ??_C@_0CI@JLGHJCBK@Illegal?5use?5of?5nonvirtual?5funct@ 10007b9c     check_code.obj
 0002:00000bc4       ??_C@_0CL@GLBBANOD@Inconsistent?5args_size?5for?5invo@ 10007bc4     check_code.obj
 0002:00000bf0       ??_C@_0DE@NNPMKFFA@Fourth?5operand?5byte?5of?5invokein@ 10007bf0     check_code.obj
 0002:00000c28       ??_C@_0ED@FJHCPNMH@invokedynamic?5bytecode?5is?5not?5s@ 10007c28     check_code.obj
 0002:00000c6c       ??_C@_0N@LDCMPJDI@Illegal?5type@ 10007c6c     check_code.obj
 0002:00000c7c       ??_C@_0BP@ODCOLLJF@Array?5with?5too?5many?5dimensions@ 10007c7c     check_code.obj
 0002:00000c9c       ??_C@_0CM@FONLGMBM@Illegal?5creation?5of?5multi?9dimen@ 10007c9c     check_code.obj
 0002:00000cc8       ??_C@_0BL@JFBHIPFA@Illegal?5dimension?5argument@ 10007cc8     check_code.obj
 0002:00000ce4       ??_C@_0BM@KCJFBPMJ@Bad?5type?5passed?5to?5newarray@ 10007ce4     check_code.obj
 0002:00000d00       ??_C@_0BO@IPLACFGP@Illegal?5local?5variable?5number@ 10007d00     check_code.obj
 0002:00000d20       ??_C@_0CJ@EJBEHDO@Quick?5instructions?5shouldn?8t?5ap@ 10007d20     check_code.obj
 0002:00000d4c       ??_C@_0BF@ONJOHFJF@Stack?5size?5too?5large@ 10007d4c     check_code.obj
 0002:00000d64       ??_C@_0BO@EMEKPNCP@Illegal?5exception?5table?5range@ 10007d64     check_code.obj
 0002:00000d84       ??_C@_0CA@FFNGPAIA@Illegal?5exception?5table?5handler@ 10007d84     check_code.obj
 0002:00000da4       ??_C@_0CH@HJMOBBMF@catch_type?5not?5a?5subclass?5of?5Th@ 10007da4     check_code.obj
 0002:00000dcc       ??_C@_0BM@DCCFFOPK@Illegal?5constant?5pool?5index@ 10007dcc     check_code.obj
 0002:00000de8       ??_C@_0BO@MHHNPBFP@Illegal?5type?5in?5constant?5pool@ 10007de8     check_code.obj
 0002:00000e08       ??_C@_0CP@OPMCNODN@Accessing?5value?5from?5uninitiali@ 10007e08     check_code.obj
 0002:00000e38       ??_C@_0CM@NPHEFIF@Cannot?5load?5return?5address?5from@ 10007e38     check_code.obj
 0002:00000e64       ??_C@_0CA@KEEKJMEB@Register?5?$CFd?5contains?5wrong?5type@ 10007e64     check_code.obj
 0002:00000e84       ??_C@_0DH@NBMNCDGB@Accessing?5value?5from?5uninitiali@ 10007e84     check_code.obj
 0002:00000ebc       ??_C@_0CI@FFLCDFOB@Register?5pair?5?$CFd?1?$CFd?5contains?5wr@ 10007ebc     check_code.obj
 0002:00000ee4       ??_C@_0CI@EGAONJHK@Constructor?5must?5call?5super?$CI?$CJ?5o@ 10007ee4     check_code.obj
 0002:00000f0c       ??_C@_0BH@CJGPGAJD@Cannot?5return?5normally@ 10007f0c     check_code.obj
 0002:00000f24       ??_C@_0CE@FBIHMBHO@Signature?5?$CFs?5has?5too?5many?5argum@ 10007f24     check_code.obj
 0002:00000f48       ??_C@_0CJ@BONIFDHI@Unable?5to?5pop?5operand?5off?5an?5em@ 10007f48     check_code.obj
 0002:00000f74       ??_C@_0CD@JACGABBD@Expecting?5to?5find?5integer?5on?5st@ 10007f74     check_code.obj
 0002:00000f98       ??_C@_0CB@NDFHAENO@Expecting?5to?5find?5float?5on?5stac@ 10007f98     check_code.obj
 0002:00000fbc       ??_C@_0CI@JKLLHFAM@Expecting?5to?5find?5object?1array?5@ 10007fbc     check_code.obj
 0002:00000fe4       ??_C@_0CO@LOLMNPNF@Expecting?5to?5find?5unitialized?5o@ 10007fe4     check_code.obj
 0002:00001014       ??_C@_0CC@GELLHINM@Expecting?5to?5find?5object?5on?5sta@ 10008014     check_code.obj
 0002:00001038       ??_C@_0DB@CONIAHKL@Expecting?5to?5find?5object?0?5array@ 10008038     check_code.obj
 0002:0000106c       ??_C@_0CC@JCNHCLNF@Expecting?5to?5find?5double?5on?5sta@ 1000806c     check_code.obj
 0002:00001090       ??_C@_0CA@LKJHBGBC@Expecting?5to?5find?5long?5on?5stack@ 10008090     check_code.obj
 0002:000010b0       ??_C@_0CJ@KKNNGPFD@Expecting?5to?5find?5array?5of?5ints@ 100080b0     check_code.obj
 0002:000010dc       ??_C@_0CK@PNKMEHAI@Expecting?5to?5find?5array?5of?5long@ 100080dc     check_code.obj
 0002:00001108       ??_C@_0CL@ICDAPAKP@Expecting?5to?5find?5array?5of?5floa@ 10008108     check_code.obj
 0002:00001134       ??_C@_0CM@MJJIIDDO@Expecting?5to?5find?5array?5of?5doub@ 10008134     check_code.obj
 0002:00001160       ??_C@_0DG@KCMJDOHN@Expecting?5to?5find?5array?5of?5obje@ 10008160     check_code.obj
 0002:00001198       ??_C@_0DG@DEMCOOEF@Expecting?5to?5find?5array?5of?5byte@ 10008198     check_code.obj
 0002:000011d0       ??_C@_0CK@HPCCGBIM@Expecting?5to?5find?5array?5of?5char@ 100081d0     check_code.obj
 0002:000011fc       ??_C@_0CL@JNPPLMFA@Expecting?5to?5find?5array?5of?5shor@ 100081fc     check_code.obj
 0002:00001228       ??_C@_0CB@NNMAOJIL@Expecting?5to?5find?5array?5on?5stac@ 10008228     check_code.obj
 0002:0000124c       ??_C@_0BC@GOJHLIAO@Internal?5error?5?$CD1@ 1000824c     check_code.obj
 0002:00001260       ??_C@_0CN@PCPDMMDA@Attempt?5to?5split?5long?5or?5double@ 10008260     check_code.obj
 0002:00001290       ??_C@_0BC@EFLKOLMN@Internal?5error?5?$CD2@ 10008290     check_code.obj
 0002:000012a4       ??_C@_0DF@NBMNBMN@Expecting?5reference?5type?5on?5ope@ 100082a4     check_code.obj
 0002:000012dc       ??_C@_0DO@OPGGFEPL@Component?5type?5of?5the?5array?5mus@ 100082dc     check_code.obj
 0002:0000131c       ??_C@_0CP@FLNEFDMF@Incompatible?5type?5for?5getting?5o@ 1000831c     check_code.obj
 0002:0000134c       ??_C@_0BN@FIPCNIKP@Bad?5access?5to?5protected?5data@ 1000834c     check_code.obj
 0002:0000136c       ??_C@_0BP@LEANFGC@Bad?5type?5in?5putfield?1putstatic@ 1000836c     check_code.obj
 0002:0000138c       ??_C@_0CB@HDEBKOAL@Can?5only?5throw?5Throwable?5object@ 1000838c     check_code.obj
 0002:000013b0       ??_C@_0CE@MGMINFON@Call?5to?5wrong?5initialization?5me@ 100083b0     check_code.obj
 0002:000013d4       ??_C@_0CP@IOILPFBI@Incompatible?5object?5argument?5fo@ 100083d4     check_code.obj
 0002:00001404       ??_C@_0CP@DFECJLLH@Incompatible?5object?5argument?5fo@ 10008404     check_code.obj
 0002:00001434       ??_C@_05KFBJCHHJ@clone@    10008434     check_code.obj
 0002:0000143c       ??_C@_0CC@PKKHICFB@Incompatible?5argument?5to?5functi@ 1000843c     check_code.obj
 0002:00001460       ??_C@_0BO@LIKPGEIF@Wrong?5return?5type?5in?5function@ 10008460     check_code.obj
 0002:00001480       ??_C@_0DA@BPKIPKAJ@Uninitialized?5object?5on?5stack?5a@ 10008480     check_code.obj
 0002:000014b0       ??_C@_0BM@KHIDEPCC@Recursive?5call?5to?5jsr?5entry@ 100084b0     check_code.obj
 0002:000014cc       ??_C@_0BC@FMKBNKIM@Internal?5error?5?$CD3@ 100084cc     check_code.obj
 0002:000014e0       ??_C@_0BA@JJLOPNCP@java?1lang?1Class@ 100084e0     check_code.obj
 0002:000014f0       ??_C@_0BM@IOMIIBEP@java?1lang?1invoke?1MethodType@ 100084f0     check_code.obj
 0002:0000150c       ??_C@_0BO@JMIOPLNI@java?1lang?1invoke?1MethodHandle@ 1000850c     check_code.obj
 0002:0000152c       ??_C@_0BF@NOENOBKG@Illegal?5signature?5?$CFs@ 1000852c     check_code.obj
 0002:00001544       ??_C@_0BC@BDOAEMEL@Internal?5error?5?$CD4@ 10008544     check_code.obj
 0002:00001558       ??_C@_0CA@OEMIIPMN@Falling?5off?5the?5end?5of?5the?5code@ 10008558     check_code.obj
 0002:00001578       ??_C@_0BP@FNHCNJPB@Multiple?5returns?5to?5single?5jsr@ 10008578     check_code.obj
 0002:00001598       ??_C@_0BP@OFOGICAN@Illegal?5return?5from?5subroutine@ 10008598     check_code.obj
 0002:000015b8       ??_C@_0CD@MGFACBCC@Inconsistent?5stack?5height?5?$CFd?5?$CB?$DN@ 100085b8     check_code.obj
 0002:000015dc       ??_C@_0BH@DHJCKLFP@Mismatched?5stack?5types@ 100085dc     check_code.obj
 0002:000015f4       ??_C@_0BC@KPLHNAK@Internal?5error?5?$CD5@ 100085f4     check_code.obj
 0002:00001608       ??_C@_0CH@LMGKOHDK@?$CIclass?3?5?$CFs?0?5method?3?5?$CFs?5signatur@ 10008608     check_code.obj
 0002:00001630       ??_C@_0BI@GMLFNJMC@?$CIclass?3?5?$CFs?0?5field?3?5?$CFs?$CJ?5@ 10008630     check_code.obj
 0002:00001648       ??_C@_0N@BACMJECO@?$CIclass?3?5?$CFs?$CJ?5@ 10008648     check_code.obj
 0002:00001660       __pDefaultRawDllMain       10008660     MSVCRT:dll_dllmain.obj
 0002:00001660       __pRawDllMain              10008660     MSVCRT:dll_dllmain.obj
 0002:00001668       __load_config_used         10008668     MSVCRT:loadcfg.obj
 0002:000017c0       ___safe_se_handler_table   100087c0     <linker-defined>
 0002:000017c4       ___volatile_metadata       100087c4     <linker-defined>
 0002:00001ac4       ___rtc_iaa                 10008ac4     MSVCRT:initsect.obj
 0002:00001ac8       ___rtc_izz                 10008ac8     MSVCRT:initsect.obj
 0002:00001acc       ___rtc_taa                 10008acc     MSVCRT:initsect.obj
 0002:00001ad0       ___rtc_tzz                 10008ad0     MSVCRT:initsect.obj
 0002:00001bb8       __IMPORT_DESCRIPTOR_jvm    10008bb8     jvm:jvm.dll
 0002:00001bcc       __IMPORT_DESCRIPTOR_KERNEL32 10008bcc     kernel32:KERNEL32.dll
 0002:00001be0       __IMPORT_DESCRIPTOR_VCRUNTIME140 10008be0     vcruntime:VCRUNTIME140.dll
 0002:00001bf4       __IMPORT_DESCRIPTOR_api-ms-win-crt-string-l1-1-0 10008bf4     ucrt:api-ms-win-crt-string-l1-1-0.dll
 0002:00001c08       __IMPORT_DESCRIPTOR_api-ms-win-crt-heap-l1-1-0 10008c08     ucrt:api-ms-win-crt-heap-l1-1-0.dll
 0002:00001c1c       __IMPORT_DESCRIPTOR_api-ms-win-crt-runtime-l1-1-0 10008c1c     ucrt:api-ms-win-crt-runtime-l1-1-0.dll
 0002:00001c30       __NULL_IMPORT_DESCRIPTOR   10008c30     jvm:jvm.dll
 0003:000000cc       ___security_cookie_complement 1000a0cc     MSVCRT:gs_cookie.obj
 0003:000000d0       ___security_cookie         1000a0d0     MSVCRT:gs_cookie.obj
 0003:000000d4       ___scrt_native_dllmain_reason 1000a0d4     MSVCRT:utility.obj
 0003:000000e0       ___isa_enabled             1000a0e0     MSVCRT:cpu_disp.obj
 0003:000000e4       ___scrt_ucrt_dll_is_in_use 1000a0e4     MSVCRT:ucrt_stubs.obj
 0003:00000408       ?__type_info_root_node@@3U__type_info_node@@A 1000a408     MSVCRT:tncleanup.obj
 0003:00000410       ?_OptionsStorage@?1??__local_stdio_printf_options@@9@4_KA 1000a410     MSVCRT:default_local_stdio_options.obj
 0003:00000418       ?_OptionsStorage@?1??__local_stdio_scanf_options@@9@4_KA 1000a418     MSVCRT:default_local_stdio_options.obj
 0003:00000420       ___scrt_current_native_startup_state 1000a420     MSVCRT:utility.obj
 0003:00000424       ___scrt_native_startup_lock 1000a424     MSVCRT:utility.obj
 0003:00000444       ___scrt_debugger_hook_flag 1000a444     MSVCRT:utility_desktop.obj
 0003:00000448       ___isa_available           1000a448     MSVCRT:cpu_disp.obj
 0003:0000044c       ___favor                   1000a44c     MSVCRT:cpu_disp.obj
 0003:00000450       ___dyn_tls_init_callback   1000a450     <common>

 entry point at        0001:00004c57

 Static symbols

 0000:ffff3000       .debug$S                   10000000     verify.exp
 0000:ffff3000       .debug$S                   10000000     vcruntime:VCRUNTIME140.dll
 0000:ffff3000       .debug$S                   10000000     vcruntime:VCRUNTIME140.dll
 0000:ffff3000       .debug$S                   10000000     vcruntime:VCRUNTIME140.dll
 0000:ffff3000       .debug$S                   10000000     vcruntime:VCRUNTIME140.dll
 0000:ffff3000       .debug$S                   10000000     vcruntime:VCRUNTIME140.dll
 0000:ffff3000       .debug$S                   10000000     vcruntime:VCRUNTIME140.dll
 0000:ffff3000       .debug$S                   10000000     vcruntime:VCRUNTIME140.dll
 0000:ffff3000       .debug$S                   10000000     vcruntime:VCRUNTIME140.dll
 0000:ffff3000       .debug$S                   10000000     vcruntime:VCRUNTIME140.dll
 0000:ffff3000       .debug$S                   10000000     ucrt:api-ms-win-crt-heap-l1-1-0.dll
 0000:ffff3000       .debug$S                   10000000     ucrt:api-ms-win-crt-heap-l1-1-0.dll
 0000:ffff3000       .debug$S                   10000000     ucrt:api-ms-win-crt-heap-l1-1-0.dll
 0000:ffff3000       .debug$S                   10000000     ucrt:api-ms-win-crt-runtime-l1-1-0.dll
 0000:ffff3000       .debug$S                   10000000     ucrt:api-ms-win-crt-runtime-l1-1-0.dll
 0000:ffff3000       .debug$S                   10000000     ucrt:api-ms-win-crt-runtime-l1-1-0.dll
 0000:ffff3000       .debug$S                   10000000     ucrt:api-ms-win-crt-runtime-l1-1-0.dll
 0000:ffff3000       .debug$S                   10000000     ucrt:api-ms-win-crt-runtime-l1-1-0.dll
 0000:ffff3000       .debug$S                   10000000     ucrt:api-ms-win-crt-runtime-l1-1-0.dll
 0000:ffff3000       .debug$S                   10000000     ucrt:api-ms-win-crt-runtime-l1-1-0.dll
 0000:ffff3000       .debug$S                   10000000     ucrt:api-ms-win-crt-runtime-l1-1-0.dll
 0000:ffff3000       .debug$S                   10000000     ucrt:api-ms-win-crt-runtime-l1-1-0.dll
 0000:ffff3000       .debug$S                   10000000     ucrt:api-ms-win-crt-runtime-l1-1-0.dll
 0000:ffff3000       .debug$S                   10000000     ucrt:api-ms-win-crt-runtime-l1-1-0.dll
 0000:ffff3000       .debug$S                   10000000     ucrt:api-ms-win-crt-runtime-l1-1-0.dll
 0000:ffff3000       .debug$S                   10000000     ucrt:api-ms-win-crt-string-l1-1-0.dll
 0000:ffff3000       .debug$S                   10000000     ucrt:api-ms-win-crt-string-l1-1-0.dll
 0000:ffff3000       .debug$S                   10000000     ucrt:api-ms-win-crt-string-l1-1-0.dll
 0000:ffff3000       .debug$S                   10000000     kernel32:KERNEL32.dll
 0000:ffff3000       .debug$S                   10000000     kernel32:KERNEL32.dll
 0000:ffff3000       .debug$S                   10000000     kernel32:KERNEL32.dll
 0000:ffff3000       .debug$S                   10000000     kernel32:KERNEL32.dll
 0000:ffff3000       .debug$S                   10000000     kernel32:KERNEL32.dll
 0000:ffff3000       .debug$S                   10000000     kernel32:KERNEL32.dll
 0000:ffff3000       .debug$S                   10000000     kernel32:KERNEL32.dll
 0000:ffff3000       .debug$S                   10000000     kernel32:KERNEL32.dll
 0000:ffff3000       .debug$S                   10000000     kernel32:KERNEL32.dll
 0000:ffff3000       .debug$S                   10000000     kernel32:KERNEL32.dll
 0000:ffff3000       .debug$S                   10000000     kernel32:KERNEL32.dll
 0000:ffff3000       .debug$S                   10000000     kernel32:KERNEL32.dll
 0000:ffff3000       .debug$S                   10000000     kernel32:KERNEL32.dll
 0000:ffff3000       .debug$S                   10000000     kernel32:KERNEL32.dll
 0000:ffff3000       .debug$S                   10000000     jvm:jvm.dll
 0000:ffff3000       .debug$S                   10000000     jvm:jvm.dll
 0000:ffff3000       .debug$S                   10000000     jvm:jvm.dll
 0000:ffff3000       .debug$S                   10000000     jvm:jvm.dll
 0000:ffff3000       .debug$S                   10000000     jvm:jvm.dll
 0000:ffff3000       .debug$S                   10000000     jvm:jvm.dll
 0000:ffff3000       .debug$S                   10000000     jvm:jvm.dll
 0000:ffff3000       .debug$S                   10000000     jvm:jvm.dll
 0000:ffff3000       .debug$S                   10000000     jvm:jvm.dll
 0000:ffff3000       .debug$S                   10000000     jvm:jvm.dll
 0000:ffff3000       .debug$S                   10000000     jvm:jvm.dll
 0000:ffff3000       .debug$S                   10000000     jvm:jvm.dll
 0000:ffff3000       .debug$S                   10000000     jvm:jvm.dll
 0000:ffff3000       .debug$S                   10000000     jvm:jvm.dll
 0000:ffff3000       .debug$S                   10000000     jvm:jvm.dll
 0000:ffff3000       .debug$S                   10000000     jvm:jvm.dll
 0000:ffff3000       .debug$S                   10000000     jvm:jvm.dll
 0000:ffff3000       .debug$S                   10000000     jvm:jvm.dll
 0000:ffff3000       .debug$S                   10000000     jvm:jvm.dll
 0000:ffff3000       .debug$S                   10000000     jvm:jvm.dll
 0000:ffff3000       .debug$S                   10000000     jvm:jvm.dll
 0000:ffff3000       .debug$S                   10000000     jvm:jvm.dll
 0000:ffff3000       .debug$S                   10000000     jvm:jvm.dll
 0000:ffff3000       .debug$S                   10000000     jvm:jvm.dll
 0000:ffff3000       .debug$S                   10000000     jvm:jvm.dll
 0000:ffff3000       .debug$S                   10000000     jvm:jvm.dll
 0000:ffff3000       .debug$S                   10000000     jvm:jvm.dll
 0000:ffff3000       .debug$S                   10000000     jvm:jvm.dll
 0000:ffff3000       .debug$S                   10000000     jvm:jvm.dll
 0000:ffff3000       .debug$S                   10000000     jvm:jvm.dll
 0000:ffff3000       .debug$S                   10000000     jvm:jvm.dll
 0000:ffff3000       .debug$S                   10000000     jvm:jvm.dll
 0000:ffff3000       .debug$S                   10000000     jvm:jvm.dll
 0000:ffff3000       .debug$S                   10000000     jvm:jvm.dll
 0001:00000000       _CCalloc                   10001000 f   check_code.obj
 0001:000000b1       _CCerror                   100010b1 f   check_code.obj
 0001:000000f7       _CCinit                    100010f7 f   check_code.obj
 0001:00000139       _CCout_of_memory           10001139 f   check_code.obj
 0001:00000158       _CFerror                   10001158 f   check_code.obj
 0001:00000513       __ck_ntohl                 10001513 f   check_code.obj
 0001:00000542       _add_to_masks              10001542 f   check_code.obj
 0001:0000060e       _check_and_push_common     1000160e f   check_code.obj
 0001:00000674       _check_and_push_malloc_block 10001674 f   check_code.obj
 0001:00000687       _check_and_push_string_utf 10001687 f   check_code.obj
 0001:0000069a       _check_register_values     1000169a f   check_code.obj
 0001:00000772       _class_name_to_ID          10001772 f   check_code.obj
 0001:00000893       _class_to_ID               10001893 f   check_code.obj
 0001:000009e3       _copy_masks                100019e3 f   check_code.obj
 0001:00000a73       _copy_stack                10001a73 f   check_code.obj
 0001:00000ac2       _cp_index_to_class_fullinfo 10001ac2 f   check_code.obj
 0001:00000b5e       _decrement_indirection     10001b5e f   check_code.obj
 0001:00000ba6       _finalize_class_hash       10001ba6 f   check_code.obj
 0001:00000c3a       _free_block                10001c3a f   check_code.obj
 0001:00000c5e       _get_result_signature      10001c5e f   check_code.obj
 0001:00000d1d       _initialize_dataflow       10001d1d f   check_code.obj
 0001:00000e65       _initialize_exception_table 10001e65 f   check_code.obj
 0001:0000103f       _instruction_length        1000203f f   check_code.obj
 0001:00001154       _isAssignableTo            10002154 f   check_code.obj
 0001:00001172       _isLegalOffset             10002172 f   check_code.obj
 0001:000011ae       _isLegalTarget             100021ae f   check_code.obj
 0001:000011d4       _load_class_global         100021d4 f   check_code.obj
 0001:0000120e       _load_class_local          1000220e f   check_code.obj
 0001:0000123c       _make_class_info           1000223c f   check_code.obj
 0001:00001258       _make_class_info_from_name 10002258 f   check_code.obj
 0001:00001271       _make_loadable_class_info  10002271 f   check_code.obj
 0001:0000128d       _merge_flags               1000228d f   check_code.obj
 0001:000012d1       _merge_fullinfo_types      100022d1 f   check_code.obj
 0001:000016c1       _merge_into_one_successor  100026c1 f   check_code.obj
 0001:000019cb       _merge_into_successors     100029cb f   check_code.obj
 0001:00001ca3       $LN82                      10002ca3     check_code.obj
 0001:00001cbf       $LN81                      10002cbf     check_code.obj
 0001:00001cf0       _merge_registers           10002cf0 f   check_code.obj
 0001:0000204d       _merge_stack               1000304d f   check_code.obj
 0001:00002126       _new_bucket                10003126 f   check_code.obj
 0001:0000218f       _object_fullinfo_to_classclass 1000318f f   check_code.obj
 0001:000021d4       _pop_and_free              100031d4 f   check_code.obj
 0001:0000220f       _pop_stack                 1000320f f   check_code.obj
 0001:00002c70       _print_CCerror_info        10003c70 f   check_code.obj
 0001:00002d5c       _push_stack                10003d5c f   check_code.obj
 0001:00003145       _read_all_code             10004145 f   check_code.obj
 0001:000031d6       _run_dataflow              100041d6 f   check_code.obj
 0001:00003339       _set_protected             10004339 f   check_code.obj
 0001:00003432       _signature_to_args_size    10004432 f   check_code.obj
 0001:000034b5       _signature_to_fieldtype    100044b5 f   check_code.obj
 0001:0000369d       _update_registers          1000469d f   check_code.obj
 0001:00003a6e       _verify_constant_pool_type 10004a6e f   check_code.obj
 0001:00003aae       _verify_method             10004aae f   check_code.obj
 0001:00003d90       _verify_opcode_operands    10004d90 f   check_code.obj
 0001:000044fc       $LN201                     100054fc     check_code.obj
 0001:00004568       $LN200                     10005568     check_code.obj
 0001:00004620       $LN202                     10005620     check_code.obj
 0001:00004917       ?dllmain_crt_dispatch@@YGHQAUHINSTANCE__@@KQAX@Z 10005917 f   MSVCRT:dll_dllmain.obj
 0001:0000496a       ?dllmain_crt_process_attach@@YAHQAUHINSTANCE__@@QAX@Z 1000596a f   MSVCRT:dll_dllmain.obj
 0001:00004a71       ?dllmain_crt_process_detach@@YAH_N@Z 10005a71 f   MSVCRT:dll_dllmain.obj
 0001:00004b21       ?dllmain_dispatch@@YAHQAUHINSTANCE__@@KQAX@Z 10005b21 f   MSVCRT:dll_dllmain.obj
 0001:00004c2c       ?dllmain_raw@@YGHQAUHINSTANCE__@@KQAX@Z 10005c2c f   MSVCRT:dll_dllmain.obj
 0001:00004c7a       ___get_entropy             10005c7a f   MSVCRT:gs_support.obj
 0001:00004d75       ?find_pe_section@@YAPAU_IMAGE_SECTION_HEADER@@QAEI@Z 10005d75 f   MSVCRT:utility.obj
 0001:000051d0       $$000000                   100061d0     MSVCRT:sehprolg4.obj
 0002:00001658       _GS_ExceptionPointers      10008658     MSVCRT:gs_report.obj
 0002:00001ad8       __sehtable$?dllmain_crt_process_attach@@YAHQAUHINSTANCE__@@QAX@Z 10008ad8     MSVCRT:dll_dllmain.obj
 0002:00001af8       __sehtable$?dllmain_crt_process_detach@@YAH_N@Z 10008af8     MSVCRT:dll_dllmain.obj
 0002:00001b20       __sehtable$?dllmain_dispatch@@YAHQAUHINSTANCE__@@KQAX@Z 10008b20     MSVCRT:dll_dllmain.obj
 0002:00001b40       __sehtable$___scrt_is_nonwritable_in_current_image 10008b40     MSVCRT:utility.obj
 0002:00001b60       .edata                     10008b60     verify.exp
 0002:00001b88       rgpv                       10008b88     verify.exp
 0002:00001b8c       rgszName                   10008b8c     verify.exp
 0002:00001b90       rgwOrd                     10008b90     verify.exp
 0002:00001b92       szName                     10008b92     verify.exp
 0002:00001b9d       $N00001                    10008b9d     verify.exp
 0002:00002176       .idata$6                   10009176     jvm:jvm.dll
 0002:000022a2       .idata$6                   100092a2     kernel32:KERNEL32.dll
 0002:0000231e       .idata$6                   1000931e     vcruntime:VCRUNTIME140.dll
 0002:00002410       .idata$6                   10009410     ucrt:api-ms-win-crt-string-l1-1-0.dll
 0002:00002432       .idata$6                   10009432     ucrt:api-ms-win-crt-heap-l1-1-0.dll
 0002:00002452       .idata$6                   10009452     ucrt:api-ms-win-crt-runtime-l1-1-0.dll
 0003:00000000       ?opcode_length@?1??instruction_length@@9@9 1000a000     check_code.obj
 0003:000000e8       _GS_ExceptionRecord        1000a0e8     MSVCRT:gs_report.obj
 0003:00000138       _GS_ContextRecord          1000a138     MSVCRT:gs_report.obj
 0003:00000404       ?__proc_attached@@3HA      1000a404     MSVCRT:dll_dllmain.obj
 0003:00000428       ?is_initialized_as_dll@@3_NA 1000a428     MSVCRT:utility.obj
 0003:00000429       ?module_local_atexit_table_initialized@@3_NA 1000a429     MSVCRT:utility.obj
 0003:0000042c       ?module_local_atexit_table@@3U_onexit_table_t@@A 1000a42c     MSVCRT:utility.obj
 0003:00000438       ?module_local_at_quick_exit_table@@3U_onexit_table_t@@A 1000a438     MSVCRT:utility.obj
 0004:00000060       $R000000                   1000b060     verify.dll.res
